:100000000C94E6000C940E010C940E010C940E015D
:100010000C940E010C940E010C940E010C940E0124
:100020000C940E010C940E010C9403040C946C04BB
:100030000C940E010C940E010C940E010C940E0104
:100040000C940E010C940E010C940E010C940E01F4
:100050000C940E010C940E010C940E010C94BB0632
:100060000C940E010C940E010C940E010C940E01D4
:100070000C940E010C940E010C940E010C940E01C4
:100080000C940E010C940E010C940E010C940E01B4
:100090000C940E010C940E010C940E010C940E01A4
:1000A0000C940E010C940E010C940E0136013901D2
:1000B00028012C0130015A015A015A013D01410128
:1000C00045014B014F015A01550100000000240079
:1000D00027002A002D003000080B00020202010058
:1000E000090400000102020000052400100105249B
:1000F000010101042402060524060001070581030D
:1001000010004009040100020A0000000705020275
:100110004000000705830240000004030904416415
:100120006166727569740043697263756974205001
:100130006C617967726F756E6400120100020000D5
:1001400000409A2311800001010203011201000204
:10015000EF0201409A231180000101020301000017
:100160000000250028002B002E00310004040404A8
:10017000040304050202020204030202020206064C
:100180000606060604040202020404040802011022
:1001900040804010204080408008020401804020C0
:1001A00010020110801020404020000000020009D1
:1001B0000F0000030401000C00000000000000001C
:1001C00000000000000000000000050711241FBE11
:1001D000CFEFDAE0DEBFCDBF11E0A0E0B1E0E2EFAB
:1001E000FFE002C005900D92A432B107D9F721E0DB
:1001F000A4E2B1E001C01D92A439B207E1F710E01A
:10020000C6EED0E004C02197FE010E94EC07C53E77
:10021000D107C9F70E941A070C94F7070C94000045
:10022000E7EBF1E04491E8E9F1E02491E9E7F1E05E
:100230009491992309F451C04423E1F150E0FA016B
:100240003197EF30F105B0F5EA5AFF4F0C94EC0707
:10025000309180003F7707C0309180003F7D03C020
:1002600030918000377F3093800024C034B53F77D1
:1002700002C034B53F7D34BD1DC0309190003F7742
:1002800007C0309190003F7D03C030919000377FD0
:10029000309390000FC03091C0003F7703C0309181
:1002A000C0003F7D3093C00005C03091C200377F51
:1002B0003093C200E92FF0E0EE0FFF1FE25AFE4F2D
:1002C000A591B4919FB7F894EC91811103C020954A
:1002D0002E2301C02E2B2C939FBF0895FC018091EB
:1002E0009301811103C08FEF9FEF08959FB7F8949A
:1002F00082E08093E9002091F20030E012161306AC
:1003000014F421E030E02115310551F084E68093AA
:1003100092018091F10080838091F200882319F08E
:100320009FBFC90108958BE68093E800F9CFCF9273
:10033000DF92EF92FF920F931F93CF93DF936C01A5
:100340007A018B01C0E0D0E0CE15DF0589F0D8013D
:100350006D918D01D601ED91FC910190F081E02D20
:10036000C6010995892B11F47E0102C02196ECCFBC
:10037000C701DF91CF911F910F91FF90EF90DF9018
:10038000CF90089580918A0181110DC082E0809301
:10039000860184E080938701109289011092880180
:1003A00081E080938A0186E891E00895CF93DF93FE
:1003B0001F92CDB7DEB76983DC01ED91FC9102801D
:1003C000F381E02D41E050E0BE016F5F7F4F099562
:1003D0000F90DF91CF91089583E08093E9008091A1
:1003E000F200882319F08AE38093E8000895CF9300
:1003F000DF931F92CDB7DEB7FC018485958597FD0D
:1004000005C02FEF3FEF358724870BC0CE01019643
:100410000E946E01019719F4898190E002C08FEF6C
:100420009FEF0F90DF91CF9108950F931F93CF937C
:10043000DF931F92CDB7DEB78C01FC0184859585D3
:1004400097FF0EC0CE0101960E946E01019719F42C
:10045000298130E002C02FEF3FEFF8013587248774
:10046000F801848595850F90DF91CF911F910F91B1
:100470000895FC018485958597FD0BC09FB7F8947E
:1004800082E08093E9008091F2009FBF90E00196A6
:1004900008959FB7F89482E08093E9008091F2007C
:1004A0009FBF90E00895409130015091310120911B
:1004B0002E0130912F0142175307B4F49091E800B8
:1004C0009570E1F39091E80092FD19C08093F100DE
:1004D000809130019091310101968F739927892B7A
:1004E00019F48EEF8093E8008091300190913101F2
:1004F0000196909331018093300181E0089580E06E
:100500000895CF92DF92EF92FF920F931F93CF93B4
:10051000DF931F92CDB7DEB7182F062FE42E862F5C
:10052000880F8E5F99830E94530283E00E945302DA
:10053000F12EC12E9981D92E8C2D8F19801798F408
:10054000F601E7FE02C0849101C080810E9453023F
:10055000182F80E00E9453028123FFEFCF1ADF0A99
:100560008111EACF01C081E00F90DF91CF911F91FF
:100570000F91FF90EF90DF90CF900895DF92EF9270
:10058000FF920F931F93CF93DF93D82E8A017B01A5
:10059000E40EF51EEB01CE15DF0571F0D7FE03C0AA
:1005A000FE01849101C088810E945302219681112D
:1005B000F2CF8FEF9FEF01C0C801DF91CF911F9164
:1005C0000F91FF90EF90DF9008950F931F93CF93BB
:1005D000DF931F92CDB7DEB782E0898342E450E01B
:1005E00068ED70E080E80E94BE020E94C201DC015A
:1005F00012960D911C9113970115110569F0D80100
:10060000ED91FC910280F381E02DBE016F5F7F4F81
:10061000C801099597FF07C089810F90DF91CF919D
:100620001F910F910895F80100851185E5CF3FB71F
:10063000F8948091290190912A01A0912B01B09109
:100640002C0126B5A89B05C02F3F19F00196A11DCE
:10065000B11D3FBFBA2FA92F982F8827820F911D58
:10066000A11DB11DBC01CD0143E0660F771F881F9E
:10067000991F4A95D1F708958F929F92AF92BF929A
:10068000CF92DF92EF92FF926B017C010E941703E1
:100690004B015C01C114D104E104F104F1F00E94AA
:1006A0001703DC01CB0188199909AA09BB09883E07
:1006B0009340A105B10570F321E0C21AD108E10809
:1006C000F10888EE880E83E0981EA11CB11CC114AD
:1006D000D104E104F10419F7DDCFFF90EF90DF9032
:1006E000CF90BF90AF909F908F9008958F929F92E0
:1006F000AF92BF92CF92DF92EF92FF920F931F9330
:10070000CF93DF935C016B018A0180910B018823F9
:1007100009F45DC080919301882309F458C0809149
:10072000350180FF05C08091E00082608093E00089
:10073000E8018AEFF82E93E0E92E2FE3822E3AE3C8
:10074000932E209709F43DC08FB7F894E092E9000A
:100750009091E80095FF06C09091F200282D291B8A
:10076000922F01C090E08FBF91110AC0FA94FF2030
:1007700071F161E070E080E090E00E943C03E1CF25
:10078000292F30E0C217D3070CF49C2F8FB7F894B1
:10079000E092E9002091E80025FF11C0292F30E008
:1007A000C21BD30BF601915020F041914093F10010
:1007B000FACFC20ED31E9091E80095FF12C08FBFF2
:1007C000C0CF84E6809334011016110644F081E016
:1007D00090E0F5019383828380E090E005C0C8013A
:1007E00003C09092E800EBCFDF91CF911F910F9162
:1007F000FF90EF90DF90CF90BF90AF909F908F9041
:1008000008950E94F2071F920F920FB60F921124C3
:100810008F939F938091E1009091E100937F90935B
:10082000E10083FF0FC01092E90091E09093EB008C
:100830001092EC0092E39093ED001092930198E0F7
:100840009093F00082FF1CC093E09093E900909198
:10085000F200992319F09AE39093E8009091340103
:10086000992329F090913401915090933401909103
:100870009201992329F090919201915090939201C5
:1008800084FF10C08091E2008E7E81608093E20040
:100890008091E1008F7E8093E100809135018E7E12
:1008A000806111C080FF11C08091E2008E7E806166
:1008B0008093E2008091E1008E7E8093E100809140
:1008C00035018E7E8160809335019F918F910F90CD
:1008D0000FBE0F901F9018951F920F920FB60F9298
:1008E0001124CF92DF92EF92FF920F931F932F93D9
:1008F0003F934F935F936F937F938F939F93AF93A8
:10090000BF93EF93FF93CF93DF93CDB7DEB76C9791
:10091000DEBFCDBF1092E9008091E80083FF0CC2DA
:10092000FE017596DE2ECF2E88E08E0F8E1729F0F1
:100930009091F10090833196F9CF84E680939201F3
:1009400082EF8093E8008D8987FF05C09091E800D1
:1009500090FFFCCF03C09EEF9093E800982F907615
:1009600009F0C5C09E892F89188D91110CC080385F
:1009700029F4809133018093F10002C01092F100BC
:100980001092F1004EC1422F50E0512B913051F4A2
:10099000811147C14130510509F043C180913301B4
:1009A0008D7F0BC0933061F481113BC14130510503
:1009B00009F037C18091330182608093330131C1E6
:1009C000953041F48091E80080FFFCCF20682093AF
:1009D000E30027C1963009F05EC0EB8CFC8C1092CE
:1009E000E9001092310110923001123091F510920D
:1009F0002F0110922E010E94E50299E0BE016F5F67
:100A00007F4FDB01E92F1D92EA95E9F799831A835D
:100A100091E09E8390EA98879AEF99872091300120
:100A200030913101275F3F4F3C832B838D831092A0
:100A3000E9001092310110923001F0922F01E09202
:100A40002E0149E050E080E00E94BE020E94E502D3
:100A5000E8C0F0922F01E0922E010E94C201DC0159
:100A60001296ED90FC901397E114F10409F4C7C0BD
:100A7000D701ED91FC910480F581E02D6D2D7C2D49
:100A8000C7010995009719F00CF0CBC0CEC0F70153
:100A9000E084F184E9CF973009F4C7C0983021F49D
:100AA00081E08093F100BDC0993009F0BAC0837035
:100AB00009F0BBC0EDE0F1E081E021E036E3908198
:100AC000992361F08093E9002093EB00919190933A
:100AD000EC003093ED008F5F873089F78EE78093CD
:100AE000EA001092EA008F89809393019AC08B8D5F
:100AF0009C8D1092E9001092310110923001909378
:100B00002F0180932E01898D81115FC08E899D896F
:100B1000913A59F4813209F088C047E050E064E02E
:100B200071E080E00E94BE027CC0913209F07DC07D
:100B3000833289F4888D90E0982F88272F89822B23
:100B4000A0E0B0E08093000190930101A093020126
:100B5000B093030166C08032B1F48091E80082FF57
:100B6000FCCFE4E0F1E087E08E0F8E1729F0909142
:100B7000F10090833196F9CF84E6809392018BEF58
:100B80008093E80006C0823209F04BC08F898093C1
:100B90000B0180913201882319F0EEEFFAE002C0D8
:100BA000E0E0F8E08091040190910501A091060138
:100BB000B0910701803B9440A105B10509F0A0C0A8
:100BC00080910B0180FF83C09BC00E94C201DC01A9
:100BD00012960D911C9113970115110531F1D80151
:100BE000ED91FC910190F081E02D6D2D7C2DC801DF
:100BF0000995811116C0F80100851185EDCF1130DE
:100C0000C1F0133091F48F89882309F455C08230E4
:100C1000E9F440E862E187E291E00E9481028823E2
:100C200021F08EEF8093E80087C081E28093EB0093
:100C300083C08B8D9C8D089711F410932D018091AA
:100C40002D01811136C06AE371E038C0813029F48A
:100C500040E868E08EE191E0E0CF833031F70E9418
:100C6000C201DC011296ED90FC9013978E010F5F8C
:100C70001F4F6801E114F10479F0D701ED91FC9167
:100C80000680F781E02DB801C7010995080F111DF5
:100C9000F701E084F184EECFD8011C92F6010190B7
:100CA0000020E9F73197BF016C197D0940E0C601CA
:100CB000B4CF6CE471E002C06AE171E061157105C6
:100CC00009F4B3CFFB01449150E080E82BCFEE3F15
:100CD0002AE0F20731F0808191819093FF0A80939E
:100CE000FE0A87E797E7918380839BE088E10FB650
:100CF000F894A895809360000FBE9093600091CF08
:100D00000FB6F894A8958091600088618093600088
:100D1000109260000FBEA895EE3F8AE0F80739F008
:100D20008091FE0A9091FF0A918380837ACF10927E
:100D3000FF0A1092FE0A75CF6C960FB6F894DEBFCC
:100D40000FBECDBFDF91CF91FF91EF91BF91AF91DA
:100D50009F918F917F916F915F914F913F912F91D3
:100D60001F910F91FF90EF90DF90CF900F900FBEEB
:100D70000F901F9018951F920F920FB60F9211248B
:100D80002F933F938F939F93AF93BF9380912501B0
:100D900090912601A0912701B09128013091240162
:100DA00026E0230F2D3720F40296A11DB11D05C0AA
:100DB00029E8230F0396A11DB11D209324018093E0
:100DC000250190932601A0932701B09328018091DB
:100DD000290190912A01A0912B01B0912C0101963B
:100DE000A11DB11D8093290190932A01A0932B018D
:100DF000B0932C01BF91AF919F918F913F912F9113
:100E00000F900FBE0F901F901895E6E3F1E013824C
:100E1000128288EE93E0A0E0B0E084839583A683FD
:100E2000B78387E191E0918380838FEF9FEF958770
:100E300084870895789484B5826084BD84B5816088
:100E400084BD85B5826085BD85B5816085BD809195
:100E50006E00816080936E0010928100809181000D
:100E60008260809381008091810081608093810005
:100E700080918000816080938000809191008260E9
:100E80008093910080919100816080939100809186
:100E900090008160809390008091C1008460809375
:100EA000C1008091C10082608093C1008091C10027
:100EB00081608093C1008091C30081608093C300F2
:100EC0008091C00082608093C0008091C2008160E8
:100ED0008093C20080917A00846080937A00809130
:100EE0007A00826080937A0080917A008E7F80936E
:100EF0007A0080917A00806880937A001092930142
:100F000010923301109235018091D7008160809357
:100F1000D70080EA8093D80089B58F7E89BD89B5D6
:100F2000826089BD09B400FEFDCF61E070E080E021
:100F300090E00E943C038091D8008F7C8061809378
:100F4000D8008091E000807F8093E0008091E100F4
:100F50008E7E8093E1008DE08093E200EEEFFFE76C
:100F6000859194918B3F9C4D19F481E080933201DF
:100F7000E8E9F1E02491E9E7F1E08491882399F030
:100F800090E0880F991FFC01E653FF4FA591B491A3
:100F9000FC01E25AFE4F859194918FB7F894EC9141
:100FA000E22BEC938FBFC0E0D0E081E00E94100103
:100FB00068EE73E080E090E00E943C0380E00E94D5
:100FC000100168EE73E080E090E00E943C032097FF
:100FD00061F30E940000E9CFEE0FFF1F0590F4912E
:100FE000E02D099481E090E0F8940C94F707F894D0
:020FF000FFCF31
:100FF200FFFFFFFF00E100000000000000C1808150
:1010020000000000000000D60176033902F7011546
:0410120002EC0100EB
:00000001FF
